S02000002E2E5C62696E5C6F70656E626C745F73746D3332663230372E73726563AC
S3150800000000800020411900088F190008911900087E
S3150800001093190008951900089719000800000000B0
S315080000200000000000000000000000009919000808
S315080000309B190008000000009D1900089F19000878
S31508000040A3190008A5190008A7190008A919000886
S31508000050AB190008AD190008AF190008B119000856
S31508000060B3190008B5190008B7190008B919000826
S31508000070BB190008BD190008BF190008C1190008F6
S31508000080C3190008C5190008C7190008C9190008C6
S31508000090CB190008CD190008CF190008D119000896
S315080000A0D3190008D5190008D7190008D919000866
S315080000B0DB190008DD190008DF190008E119000836
S315080000C0E3190008E5190008E7190008E919000806
S315080000D0EB190008ED190008EF190008F1190008D6
S315080000E0F3190008F5190008F7190008F9190008A6
S315080000F0FB190008FD190008FF190008011A000875
S31508000100031A0008051A0008071A0008091A000841
S315080001100B1A00080D1A00080F1A0008111A000811
S31508000120131A0008151A0008171A0008191A0008E1
S315080001301B1A00081D1A00081F1A0008211A0008B1
S31508000140231A0008251A0008271A0008291A000881
S315080001502B1A00082D1A00082F1A0008311A000851
S31508000160331A0008351A0008371A0008391A000821
S315080001703B1A00083D1A00083F1A0008411A0008F1
S31508000180431A000810B5054C237833B9044B13B14C
S315080001900448AFF300800123237010BD84000020BB
S315080001A00000000090500008084B10B51BB1084924
S315080001B00848AFF300800848036803B910BD074B29
S315080001C0002BFBD0BDE81040184700BF0000000018
S315080001D088000020905000088400002000000000DD
S315080001E0154B002B08BF134B9D46A3F5803A0021FB
S315080001F08B460F461348144A121A04F095FA0F4B09
S31508000200002B00D098470E4B002B00D098470020B3
S31508000210002104000D000D48002802D00C48AFF359
S31508000220008004F05BFA2000290000F0FFFF04F0CC
S3150800023041FA00BF0000080000800020000000000E
S315080002400000000084000020F40F002000000000D9
S315080002500000000008B500F0D5F84FF40051034837
S3150800026000F026FE003018BF012008BD0008024035
S3150800027008B5642000F094F808BD00BF08B500F082
S3150800028095F808BD00B589B020220021684604F01B
S315080002904BFA6946094803F041FF40B9009B43B150
S315080002A09DF8080080F01000C0F3001002E000205E
S315080002B000E0002009B05DF804FB00BF54470008C1
S315080002C0004870475447000808B50748002380F8D7
S315080002D024320A22054903F07FFB18B90122024B92
S315080002E083F8242208BD00BFA0000020704700083C
S315080002F070B50E4B93F82432012B02D10B4803F04C
S3150800030037FE01F0E7FB00F16406094D402403E0DF
S3150800031001F0E0FB864205D32146284600F012FF8D
S315080003200028F5D0034803F01BFF70BDA00000208D
S31508000330004800405447000808B5044B93F8243297
S31508000340012B02D1014803F013FE08BDA0000020CE
S3150800035070B50646104B93F82432012B0AD10E4984
S3150800036003F0A0FF002805DA0B48002380F82432A2
S3150800037003F0FEFD317871B1084C8025204600F067
S31508000380D9FE2946204600F0DDFE0028F9D016F8E9
S31508000390011F0029F2D170BDA000002000480040CE
S315080003A0014B1880704700BFCC02002008B501F049
S315080003B091FB104B1B6898421AD30F4B1B7843B915
S315080003C001220D4B1A704FF480710C4800F076FD2F
S315080003D007E00022084B1A704FF48071074800F0B6
S315080003E06FFD01F077FB064B1B881844014B18601C
S315080003F008BD00BFC8020020CE020020001402403B
S31508000400CC02002008B54FF48071024800F058FD70
S3150800041008BD00BF0014024038B50146074800F081
S3150800042005FE064D01242146284600F00FFE002849
S31508000430F9D0024800F0F6FDC0B238BD003C0040D5
S3150800044038B54FF4FA72084B1A60FF241D46204649
S31508000450FFF7E2FFFF2802D02B68002BF7D1FF2811
S3150800046014BF0020012038BDD402002008B504219D
S31508000470034800F023FDFF20FFF7CEFF08BD00BFAD
S31508000480000C024010B50421074800F019FDFF20B2
S31508000490FFF7C2FFFFF7D4FF18B90446FFF7E6FFD8
S315080004A000E00124204610BD000C024038B5044681
S315080004B00D4610F0800F07D000213720FFF7F6FF12
S315080004C001283AD804F07F04FFF7D0FFFFF7DAFFD8
S315080004D048B344F04000FFF79FFF280EFFF79CFF44
S315080004E0C5F30740FFF798FFC5F30720FFF794FF0A
S315080004F0E8B2FFF791FFE4B1082C16D00120FFF708
S315080005008BFF0C2C02D1FF20FFF786FF0A24FF255C
S315080005102846FFF781FF10F0800F0ED0631E13F0F8
S31508000520FF04F5D138BDFF2038BD8720FFF774FFDB
S31508000530ECE79520FFF770FFE8E738BD38B50546C4
S315080005400C46FFF77DFF034618B32046FFF764FF06
S31508000550FD2C1DD0AC1C05F2022514F8020CFFF781
S315080005605BFF14F8010CFFF757FF0234AC42F4D1D5
S31508000570FF20FFF751FFFF20FFF74EFFFF20FFF791
S315080005804BFF00F01F00052814BF0023012300E0DD
S315080005900123184638BD00BFF8B504460D46642247
S315080005A0144B1A60FF261F463046FFF735FFFF2813
S315080005B004D13B68002BF7D10020F8BDFE2816D1E0
S315080005C00234FF263046FFF727FF04F8020C3046B0
S315080005D0FFF722FF04F8010C0234023DF2D1FF2096
S315080005E0FFF71AFFFF20FFF717FF0120F8BD0020CD
S315080005F0F8BD00BFD0020020002840F06A81BA4B3F
S315080006001B7813F0020F03D0B74B1878C0B27047A7
S315080006102DE9F0478AB00121082000F0B9FC012134
S31508000620042000F0B5FC01214FF4004000F0BEFCA8
S315080006304FF00409CDF8009002268DF805600127D1
S315080006408DF8047000248DF807408DF80640DFF811
S31508000650A0826946404600F0E3FB4946404600F062
S315080006602DFCA24D06220A21284600F02BFC062264
S315080006700B21284600F026FC06220C21284600F00D
S3150800068021FC4FF4E05300938DF804608DF8056063
S315080006908DF806408DF807606946284600F0C0FBCD
S315080006A0ADF810404FF48273ADF81230ADF814402F
S315080006B0ADF81640ADF818404FF40073ADF81A308F
S315080006C03023ADF81C30ADF81E400723ADF82030B6
S315080006D0DFF828A204A9504600F076FC21465046C9
S315080006E000F0A6FC3946504600F08EFC49464046C6
S315080006F000F0E4FB8DF80D608DF80C708DF80F4056
S315080007008DF80E404FF480540AA941F8204D28462A
S3150800071000F086FB2146284600F0D0FB0A275446FF
S315080007203146204600F092FC0028F9D0FF212046E9
S3150800073000F07CFC01252946204600F087FC0028AD
S31508000740F9D0013FECD14FF48053029302238DF880
S315080007500C308DF80D3000248DF80E408DF80F30D2
S3150800076002A9624800F05CFB0421614800F0A8FB7E
S3150800077021462046FFF79AFE012840F0AC804FF448
S315080007807A725C4B1A604FF4D5710820FFF78EFE1B
S31508000790012842D109AD0AAE2C46FF273846FFF795
S315080007A03BFE04F8010BB442F8D19DF82630012B24
S315080007B040F091809DF82730AA2B40F08C80DFF816
S315080007C034814FF08047A924D8F800302BB1394638
S315080007D02046FFF76BFE0028F6D1464B1B68002B18
S315080007E079D000213A20FFF761FE002873D1FF2453
S315080007F02046FFF711FE05F8010BB542F8D19DF822
S31508000800243003F04003DBB2002B14BF0C22042271
S31508000810394B1A60FFF72AFE23E00021A920FFF7CB
S3150800082045FE012887BF01273D460227A925314CE9
S31508000830002623682BB131462846FFF737FE0028E5
S31508000840F7D12C4B1B68002B45D04FF400711020B4
S31508000850FFF72CFE00283ED1274B1F60FFF706FE48
S3150800086077B3214A137803F0FE031370234D002152
S31508000870284600F0C9FB0024ADF810404FF48273F7
S31508000880ADF81230ADF81440ADF81640ADF8184082
S315080008904FF40073ADF81A30ADF81C40ADF81E40A1
S315080008A00723ADF8203004A9284600F08DFB214621
S315080008B0284600F0BDFB0121284600F0A5FB04E010
S315080008C0094A137843F001031370074B1878C0B22E
S315080008D007E0012070470022074B1A60FFF7C6FDA4
S315080008E0EEE70AB0BDE8F0870000002000080240E5
S315080008F0000C0240D0020020D8020020003C004034
S3150800090018B9034B1878C0B270470120704700BF6A
S315080009100000002000283BD170B50D461C46002B70
S3150800092038D01E4B1B7813F0010F35D11C4B1B68B2
S3150800093013F0080F08BF5202012C0DD111461120E1
S31508000940FFF7B4FDF0B94FF400712846FFF724FE0F
S31508000950B0FA80F4640915E011461220FFF7A6FDE7
S3150800096080B94FF4007631462846FFF715FE28B1C0
S3150800097005F50075601E10F0FF04F4D100210C2067
S31508000980FFF794FDFFF772FD201C18BF012070BD0C
S3150800099004207047042070BD032070BD00000020AD
S315080009A0D8020020002849D170B50E4615461C46C7
S315080009B0002B45D0254B1B7813F0010F42D1234B52
S315080009C01B7813F0040F3FD1214B1B6813F0080F57
S315080009D008BF5502012C0CD129461820FFF766FDE1
S315080009E030BBFE213046FFF7A9FDB0FA80F4640952
S315080009F01EE013F0060F03D021469720FFF756FD99
S31508000A0029461920FFF752FD90B9FC25294630469C
S31508000A10FFF794FD28B106F50076601E10F0FF0476
S31508000A20F4D1FD210020FFF789FD002808BF012425
S31508000A30FFF71CFD201C18BF012070BD042070475D
S31508000A40042070BD032070BD022070BD0000002088
S31508000A50D8020020002840F02681964B1B7813F018
S31508000A60010F40F0228170B584B014460E2900F2B9
S31508000A70FF80DFE811F00F001500FD005C00FD00A7
S31508000A80FD00FD00FD00FD00FD00B700BC00CA002A
S31508000A90D700E800FFF7F6FCB0FA80F46409FEE038
S31508000AA000210920FFF702FD002840F0E38010210D
S31508000AB06846FFF771FD002800F0DE809DF80030DB
S31508000AC09B09012B10D19DF808209DF8093003EBEE
S31508000AD002229DF807301B0403F47C1301331344E8
S31508000AE09B0223600024DAE09DF808209DF8073071
S31508000AF09B0003EB92129DF806309B0203F44063B9
S31508000B00134401339DF8052002F00F029DF80A10E0
S31508000B1002EBD112911C9DF80920520002F0060240
S31508000B200A44D2B2093A934023600024B7E0624BE4
S31508000B301B6813F0040F21D000218D20FFF7B6FCA7
S31508000B40002840F09B80FF20FFF766FC10216846CE
S31508000B50FFF722FD002800F093803025FF26304657
S31508000B60FFF75AFC6B1E13F0FF05F8D19DF80A3003
S31508000B701A09102393402360002490E000210920DD
S31508000B80FFF794FC00287DD110216846FFF704FD85
S31508000B90002879D0484B1B6813F0020F11D09DF836
S31508000BA00A305B0003F07E039DF80B2003EBD2139B
S31508000BB001339DF80D209209013A934023600024E1
S31508000BC06DE09DF80B10CB0003F0180303EB5111F1
S31508000BD09DF80A20C2F38402531C01FB03332360E9
S31508000BE000245CE0344B1B681370002457E0002196
S31508000BF00920FFF75BFC002848D110212046FFF7A3
S31508000C00CBFCB0FA80F4640949E000210A20FFF71A
S31508000C104DFCE8BB10212046FFF7BEFCB0FA80F475
S31508000C2064093CE000213A20FFF740FC90BB651EB2
S31508000C300334FF263046FFF7EFFB05F8010FAC42F9
S31508000C40F8D100242BE01C4B1B6813F0040F23D0AB
S31508000C5000218D20FFF72AFC00BBFF20FFF7DCFBF5
S31508000C6040212046FFF798FCB0FA80F4640916E0A4
S31508000C70042414E0012412E0012410E001240EE00B
S31508000C8001240CE001240AE0012408E0012406E01E
S31508000C90012404E0012402E0012400E00124FFF716
S31508000CA0E5FB204603E0042070470320704704B0A4
S31508000CB070BD00BF00000020D80200200048704721
S31508000CC00000AA42054B1B69002B05DA034B044AB0
S31508000CD05A6002F188325A60704700BF003C0240F1
S31508000CE023016745024A136943F0004313617047BD
S31508000CF0003C0240014BD860704700BF003C0240F0
S31508000D000E4BDB6813F4803F12D10C4BDB6813F0F3
S31508000D10100F0FD1094BDB6813F0EF0F0CD1074BFF
S31508000D20DB6803F00203002B14BF07200820704776
S31508000D30012070470520704706207047003C024096
S31508000D4000B583B008238DF80730FFF7D9FF8DF873
S31508000D5007009DF80730DBB2012B08D1FFF7D0FF5B
S31508000D608DF807009DF80730DBB2012BF6D09DF809
S31508000D70070003B05DF804FB70B5054641B10129CB
S31508000D8008D002290CBF4FF400764FF4407603E0F2
S31508000D90002601E04FF48076FFF7D2FF08281ED11F
S31508000DA00F4C236923F44073236123691E4326618C
S31508000DB0236923F0F8032361236943F002031D43E3
S31508000DC02561236943F480332361FFF7B9FF23695B
S31508000DD023F002032361236923F0F803236170BD1E
S31508000DE0003C024070B505460E46FFF7A9FF0828E5
S31508000DF013D10A4C236923F440732361236943F40E
S31508000E0000732361236943F0010323612E60FFF712
S31508000E1097FF236923F00103236170BD003C02405C
S31508000E20F0B500230125032605FA03F20C68A24350
S31508000E3039D102685C0006FA04F7FF433A400260BB
S31508000E40026891F804E00EFA04FE4EEA0202026015
S31508000E500A79013AD2B2012A17D882681740876000
S31508000E6087684A79A2403A43826047689AB205FA87
S31508000E7002FE27EA0E074760D0F804E08F7907FAE2
S31508000E8002F292B242EA0E024260C7689AB2520071
S31508000E9006FA02F227EA0202C260C268CF7907FAA6
S31508000EA004F41443C4600133102BBDD1F0BD00BF58
S31508000EB00369194214BF0120002070470183704757
S31508000EC04183704710B401F007039B00C90800EB83
S31508000ED08100046A0F21994024EA01010162016A2E
S31508000EE09A400A43026210BC704700BF10B4244BF4
S31508000EF09B6803F00C03042B05D0082B06D00BBB0C
S31508000F00204B036020E0204B03601DE01C4B5A6811
S31508000F105B6803F03F0312F4800F194A5268C2F364
S31508000F20881214BF18491749B1FBF3F303FB02F201
S31508000F30134B5B68C3F3014301335B00B2FBF3F366
S31508000F40036001E00F4B03600D4CA368C3F3031362
S31508000F500E49CB5CDAB20368D3404360A268C2F399
S31508000F6082228A5CD2B223FA02F28260A268C2F3B3
S31508000F7042328A5CD2B2D340C36010BC704700BF0D
S31508000F80003802400024F40040787D010400002067
S31508000F9021B1054B1A6B104318637047024A136B4D
S31508000FA023EA0000106370470038024021B1054B60
S31508000FB01A6C104318647047024A136C23EA00003F
S31508000FC0106470470038024010B4038803F4415493
S31508000FD00A884B8813438A881343CA8813430A89A5
S31508000FE013434A8913438A891343CA8913432343FC
S31508000FF09BB20380838B23F400631B041B0C83833F
S315080010000B8A038210BC704729B103889BB243F050
S31508001010400303807047038823F040031B041B0C1E
S3150800102003807047808980B2704700BF818170470E
S3150800103029B103889BB243F40053038070470388A1
S3150800104023F400531B041B0C0380704703891942C1
S3150800105014BF01200020704730B585B004460D4600
S31508001060038A9BB223F44053CA88134303828389B5
S315080010709BB223F4B05323F00C0289882B890B43C7
S3150800108069890B439BB213438381838A9BB223F4FA
S315080010904073AA89134383826846FFF727FF1C4BD0
S315080010A09C4203D003F580639C4201D1039B00E078
S315080010B0029BA28912F4004F03EB830303EB83031D
S315080010C0296814BF49008900B3FBF1F1114BA3FB52
S315080010D0012358090501642300FB1313A28912F49E
S315080010E0004F09D0D90032310A4AA2FB0131C1F3B7
S315080010F0421242EA050307E01B013233054AA2FB06
S315080011000323C3F343132B439BB2238105B030BD9E
S31508001110001001401F85EB5129B183899BB243F426
S31508001120005383817047838923F400531B041B0CE7
S3150800113083817047C1F30801818070478088C0F3B6
S31508001140080070470388194214BF01200020704721
S3150800115082B0314B1A6842F001021A600021996088
S315080011601A6822F0847222F480321A602B4A5A6076
S315080011701A6822F480221A60D960009101911A68CF
S3150800118042F480321A601A46136803F40033019356
S31508001190009B01330093019B1BB9009BB3F5C06FFD
S315080011A0F2D11D4B1B6813F4003F14BF0123002323
S315080011B00193019B012B29D1174B9A689A609A686B
S315080011C042F400429A609A6842F4A0529A60144A1D
S315080011D05A601A6842F080721A601A46136813F049
S315080011E0007FFBD040F203720E4B1A60A3F58063B2
S315080011F09A6822F003029A609A6842F002029A609C
S315080012001A46936803F00C03082BFAD14FF00062D4
S31508001210054B9A6002B0704700380240103000242F
S31508001220193C4005003C024000ED00E080B582B064
S3150800123001212020FFF7ACFE01210420FFF7A8FEBC
S3150800124001214FF48020FFF7B1FE01210820FFF7A6
S315080012509FFE4FF48078CDF8008000268DF8066052
S3150800126001258DF8075002248DF805408DF80450A5
S315080012702F4F69463846FFF7D3FD41463846FFF7F4
S315080012801FFE8DF804608DF807604FF40053009335
S3150800129069462848FFF7C4FDA7F500670722082115
S315080012A03846FFF70FFE072209213846FFF70AFEE0
S315080012B08DF806608DF807508DF80440CDF800804B
S315080012C08DF8054069463846FFF7AAFD8DF80440B3
S315080012D04FF40073009369463846FFF7A1FD294687
S315080012E02046FFF755FEA7F500670922082138466C
S315080012F0FFF7E8FD092211463846FFF7E3FD4FF4EC
S31508001300407300938DF804408DF805408DF806600B
S315080013108DF8075069463846FFF782FD29464FF093
S315080013200070FFF743FE00F0D9FC00F0E7FCFCE78D
S315080013300014024000080240F8B54A4A02F1240E99
S3150800134000264FF4FA7747F23050157854782B195F
S3150800135003FB077390FBF3F103FB110139B990FB0B
S31508001360F3F39EB2731E9BB2B3F5806F03D30232BA
S315080013709645EAD16EE03C4B00225A611A6842F45F
S3150800138000421A601B6813F4004F06D0364F00F06F
S3150800139031FD3B6813F4004FF9D1334B1A6822F03C
S315080013A002021A601A6842F001021A605B6813F0BA
S315080013B0010F06D12C4F00F01DFD7B6813F0010FBD
S315080013C0F9D0013D013C240544EA0545731E1D4339
S315080013D0254AD561136823F001031360536813F097
S315080013E0010F06D0144600F005FD636813F0010FDF
S315080013F0F9D11D4BD3F8002242F00102C3F80022AE
S31508001400D3F81C2222F00102C3F81C22D3F80C22BE
S3150800141042F00102C3F80C220022C3F84022C3F8A6
S315080014204422D3F8042222F00102C3F80422D3F896
S31508001430142222F00102C3F81422D3F81C2242F027
S315080014400102C3F81C22D3F8002222F00102C3F8D5
S315080014500022F8BDEC21054800F00AFC00252C46C0
S3150800146089E700BFA84700080064004080470008D5
S3150800147038B504460D46224B9B6813F0806F04D19D
S315080014804FF4A0711F4800F0F3FB1D4BD3F88021E1
S3150800149002F00102C3F88021D3F8802142F07C4291
S315080014A042F40012C3F88021C3F88451E078A17889
S315080014B00A0442EA006122780A43617842EA012274
S315080014C0C3F88821E079A1790A0442EA0061227901
S315080014D00A43617942EA0122C3F88C21D3F88021B4
S315080014E042F00102C3F880219B6813F0806F06D191
S315080014F0034C00F07FFCA36813F0806FF9D038BD69
S3150800150000640040804700081B4BDB6813F0030F9C
S315080015102FD0194BD3F8B02140F26763B3EB525F73
S3150800152020D1154BD3F8B8210270D3F8B821120A86
S315080015304270D3F8B821120C8270D3F8B821120E73
S31508001540C270D3F8BC210271D3F8BC21120A4271C9
S31508001550D3F8BC21120C8271D3F8BC311B0EC371AF
S31508001560012000E00020044AD36843F02003D3603A
S3150800157070470020704700BF0064004008B500F0BF
S31508001580DBF908BD10B500F06DFAA0B1FEF762FEF2
S3150800159088B100F0EBFB00F089FA00F067FA20F05A
S315080015A0604020F07F00044B186000F05FFA446842
S315080015B000F0C4F9A04710BD08ED00E072B170B59F
S315080015C00D46561EB6B2441E064415F8013B04F8ED
S315080015D0013F00F00FFCB442F7D170BD704700BF61
S315080015E070B506460B4D002400F004FC2B68B34288
S315080015F00AD86A6813449E4206D204EB4401054B96
S3150800160003EB8101087A70BD01340C35062CEBD149
S31508001610FF2070BDE44700082DE9F84380460068BE
S31508001620FFF7DEFFFF282FD0FFF74CFBF320FFF76D
S3150800163061FBFFF765FB012818BF002404D1FFF7FB
S3150800164051FB0020BDE8F883D8F8007004EB0709C1
S31508001650251D58F8056000F0CDFB31464846FFF7D2
S31508001660C1FB082808D1E3599E4207D12C46B5F597
S31508001670007FE9D1012402E0002400E00024FFF7FE
S3150800168031FB2046BDE8F8830020BDE8F88300BF9B
S3150800169038B50D46114B984207D00446104B99426F
S315080016A008D0FFF7B9FF08B911E00E4CC5F30803D7
S315080016B07BB900E0094C2368AB420CD0204640F8C1
S315080016C0045B4FF400722946FFF778FF03E0002019
S315080016D038BD002038BD204638BD00BFDC020020DA
S315080016E000800008E00400202DE9F04106460C467B
S315080016F017461D4621F4FF7828F001080368B3F160
S31508001700FF3F06D140F8048B4FF400724146FFF7BD
S3150800171055FF3368984505D041463046FFF7B8FF70
S315080017200646E0B13368E41A3444043408F5007810
S3150800173000F060FB331DE31AB3F5007F06D341467C
S315080017403046FFF7A5FF064660B1041D17F8013BB2
S3150800175004F8013B013DEBD10120BDE8F0810020F2
S31508001760BDE8F0810020BDE8F08100BF4FF0FF33EF
S31508001770024A1360024A1360704700BFE004002063
S31508001780DC02002070B504460D461646FFF728FF12
S31508001790FF2814D0681E2044FFF722FFFF2810D028
S315080017A024F4FF7323F00103074A93422B4632467B
S315080017B021460CBF05480648FFF796FF70BD002076
S315080017C070BD002070BD00BF00800008DC0200204C
S315080017D0E0040020F8B506460D46FFF701FF04466B
S315080017E0681E3044FFF7FCFE84422AD80546A31E2D
S315080017F0DBB2FC2B27D8072827D8FFF763FAF32094
S31508001800FFF778FAFFF77CFA012803D1FFF76AFA9F
S315080018100020F8BD0E4F022600F0ECFA314637F8E4
S315080018201400FFF7A9FA082803D0FFF75BFA00208F
S31508001830F8BD0134E4B2A542EED2FFF753FA01200F
S31508001840F8BD0020F8BD0020F8BD0020F8BD00BF97
S31508001850CC470008114B1B68B3F1FF3F18D000B501
S3150800186083B00E4B59689A681144DA6811441A69AC
S3150800187011445A6911449A691144DA698B185B4212
S3150800188002AA42F8043D04210548FFF77BFF01E060
S315080018900120704703B05DF804FB00BFDC0200209E
S315080018A0848100080D4B1A6804331B6813440C4ADC
S315080018B0126813440B4A126813440B4A11680B4406
S315080018C0043212681A44094B1B681344084A126802
S315080018D0D3420CBF01200020704700BF00800008DB
S315080018E0088000080C80000810800008188000088E
S315080018F08481000808B50C4B1B68B3F1FF3F04D080
S315080019000948FFF789FE034660B1084B1B68B3F127
S31508001910FF3F06D00548FFF77FFE031C18BF0123CB
S3150800192000E00123184608BDDC020020E004002080
S31508001930004870470080000872B6704762B6704764
S3150800194007498D460749084A084B9A42BEBF51F8CF
S31508001950040B42F8040BF8E705488047054800479A
S31508001960008000209C500008000000208400002011
S3150800197051110008E10100083249334A002301E009
S3150800198041F8043B9142FBD3FFF750FCFEE7FEE724
S31508001990FEE7FEE7FEE7FEE7FEE7FEE7FEE7FEE711
S315080019A0FEE7FEE7FEE7FEE7FEE7FEE7FEE7FEE701
S315080019B0FEE7FEE7FEE7FEE7FEE7FEE7FEE7FEE7F1
S315080019C0FEE7FEE7FEE7FEE7FEE7FEE7FEE7FEE7E1
S315080019D0FEE7FEE7FEE7FEE7FEE7FEE7FEE7FEE7D1
S315080019E0FEE7FEE7FEE7FEE7FEE7FEE7FEE7FEE7C1
S315080019F0FEE7FEE7FEE7FEE7FEE7FEE7FEE7FEE7B1
S31508001A00FEE7FEE7FEE7FEE7FEE7FEE7FEE7FEE7A0
S31508001A10FEE7FEE7FEE7FEE7FEE7FEE7FEE7FEE790
S31508001A20FEE7FEE7FEE7FEE7FEE7FEE7FEE7FEE780
S31508001A30FEE7FEE7FEE7FEE7FEE7FEE7FEE7FEE770
S31508001A40FEE7FEE784000020F40F002008B5FFF744
S31508001A508DFE08BD08B5FFF795FE08BD08B5FFF76A
S31508001A60B9FE08BD08B5FFF71DFF08BD08B5FFF7A5
S31508001A705FFF08BD08B5FFF7EDFE034610B1FFF797
S31508001A8039FF0346184608BD054B00221A6005496A
S31508001A9059609A6005211960034B1A60704700BFA8
S31508001AA010E000E0BFD40100E40600200022014B4C
S31508001AB01A60704710E000E0044B1B6813F4803F7F
S31508001AC003D0034A136801331360704710E000E03F
S31508001AD0E406002008B5FFF7EFFF014B186808BDBC
S31508001AE0E406002038B5044680210A48FFF72AFB99
S31508001AF068B121460748FFF71DFB064D802421469D
S31508001B002846FFF71FFB0028F9D0012038BD002022
S31508001B1038BD00BF0048004010B5044620210648DD
S31508001B20FFF710FB012805D10348FFF707FB2070D4
S31508001B30012010BD002010BD0048004010B584B03B
S31508001B404FF4614300930023ADF80430ADF8063036
S31508001B50ADF80830ADF80C300C23ADF80A30054C5A
S31508001B6069462046FFF778FA01212046FFF7D4FA9E
S31508001B7004B010BD00480040F8B505460C4640299B
S31508001B8003D97521114800F073F82046FFF7AAFF1C
S31508001B90012803D079210D4800F06AF8A3B29BB159
S31508001BA06C1E013B9BB21D44084F822600F022F9A9
S31508001BB014F8010FFFF796FF012803D0314638467F
S31508001BC000F056F8AC42F1D1F8BD00BF2C48000829
S31508001BD038B5224B1C789CB92148FFF79DFF012890
S31508001BE039D11F4B1B78002B30D0FFF773FF1D4BE5
S31508001BF0186000221C4B1A700122184B1A702AE032
S31508001C000546194B1878194B1844FFF785FF044603
S31508001C10012810D1144B1A780132D2B21A70104B1F
S31508001C201B78934214D111492846FFF7C7FC0022B6
S31508001C300A4B1A700FE0FFF74DFF0A4B1B68643317
S31508001C40984207D90024054B1C7004E01C4602E0A4
S31508001C50002400E00024204638BD00BF2A070020E3
S31508001C60E80600202C07002029070020E9060020A6
S31508001C7008B500F0BFF8FCE708B500F0B3F801288E
S31508001C8016D000F03FF998B10A4B1B78012B0FD1FB
S31508001C90FFF720FF084B1B6803F5FA73984207D332
S31508001CA00022044B1A7000F035F908B9FFF76AFCF0
S31508001CB008BD00BF300700203407002008B5012200
S31508001CC0044B1A70FFF706FF034B1860FFF7D4FFA3
S31508001CD008BD00BF300700203407002008B5FFF70D
S31508001CE04DFC00F083F8FFF7CFFEFFF7AFFE00F0DC
S31508001CF0F5F800F00FF8FFF7E1FF08BD08B500F0AA
S31508001D0079F8FFF7D9FE00F023FA00F013F8FFF789
S31508001D10B3FF08BD10B502F01FFBFFF70DFB044C1F
S31508001D2001232370FFF70AFF0023237010BD00BFAD
S31508001D301400002008B50B48FFF7E6FB012805D17B
S31508001D400122094B1A70074802F024FB0548FFF7E1
S31508001D503FFF012805D10022034B1A70014802F003
S31508001D6019FB08BD3807002014000020704700BF83
S31508001D7038B504460D46084B1B78012B02D1C9B26B
S31508001D80FFF776FB044B1B781BB9E9B22046FFF731
S31508001D90F3FE02F0F7FA38BD14000020074B1B7853
S31508001DA0022B06D0032B06D0012B0CBF082040209F
S31508001DB07047002070470020704700BF14000020BD
S31508001DC0074B1B78022B06D0032B06D0012B0CBF22
S31508001DD0082040207047002070470020704700BF49
S31508001DE01400002008B502F0C5FA08BD08B5FEF7CC
S31508001DF03FFA08BD08B5FEF741FA08BD00F00F0323
S31508001E00092802D903F13700704703F13000054B62
S31508001E101B6803445B7803F00303022B08BF2038D2
S31508001E20C0B270471800002038B505460C460009B0
S31508001E30FFF7E4FF207005F00F00FFF7DFFF607083
S31508001E400023A370204638BD10B4034602460C484A
S31508001E500131A0FB0242D208FAD100220A70084CCE
S31508001E60A4FB0302D20802EB8200A3EB4003303343
S31508001E7001F8013D1346002AF2D1084610BC704706
S31508001E80CDCCCCCC70B4144B1E68441E451C002027
S31508001E9014F8013FF218517801F00301022908BF2E
S31508001EA0203BDBB2A3F13002D2B2162A0FD8A3F137
S31508001EB03A01C9B206290CD9092A84BF373BDAB2D6
S31508001EC002EB001303F0FF00AC42E1D102E0002070
S31508001ED000E0002070BC70471800002008B50020FC
S31508001EE0054B1870054901F065FD18B177210448BE
S31508001EF0FFF7BEFE08BD00BFB8070020C4070020D4
S31508001F0058480008024B1878B0FA80F04009704724
S31508001F10B807002008B5FFF765FF01280AD0084B67
S31508001F201B784BB9FEF7AEF9012807D10122044BFD
S31508001F301A7008BD002008BD002008BD002008BD95
S31508001F40B80700200378114A1168CA18527802F0B7
S31508001F500302022A08BF203B532B0ED143781944AB
S31508001F604A7812F0040F0AD0312B0AD0322B0AD045
S31508001F70332B0CBF02200320704703207047032031
S31508001F807047002070470120704700BF18000020E6
S31508001F9070B506460230FFF775FF054684B204366B
S31508001FA03046FFF76FFF2844C5B2013CA4B202369B
S31508001FB0012CF5D83046FFF765FFED43EDB28542B3
S31508001FC014BF0020012070BD2DE9F04104461646D5
S31508001FD0884601B120B940F233215C48FFF748FE34
S31508001FE02046FFF7AFFF0546032800F092802046FB
S31508001FF0FFF7CEFF002800F08F80012D28D015B1FD
S31508002000022D52D08CE0A01CFFF73CFF0746201D8E
S31508002010FFF738FF0502C8F80050A01DFFF732FF8A
S315080020202844C8F800000834F81E07B2002E7AD0F3
S31508002030B846002F7ADD00252046FFF723FF7055A6
S3150800204002340135ADB24545F6DB3846BDE8F081C8
S31508002050A01CFFF717FF0746201DFFF713FF05040F
S31508002060C8F80050A01DFFF70DFF05EB0025C8F8BE
S31508002070005004F10800FFF705FF2844C8F80000DF
S315080020800A34381F07B2002E53D0B846002F53DD46
S3150800209000252046FFF7F6FE705502340135ADB22D
S315080020A04545F6DB3846BDE8F081A01CFFF7EAFE99
S315080020B00746201DFFF7E6FE0506C8F80050A01DD6
S315080020C0FFF7E0FE05EB0045C8F8005004F10800EC
S315080020D0FFF7D8FE05EB0025C8F8005004F10A0002
S315080020E0FFF7D0FE2844C8F800000C34781F07B262
S315080020F02EB3B846002F25DD00252046FFF7C2FE81
S31508002100705502340135ADB24545F6DB3846BDE8B3
S31508002110F0810020BDE8F0814FF0FF30BDE8F08186
S315080021200020BDE8F0813846BDE8F0813846BDE8B4
S31508002130F0813846BDE8F0813846BDE8F08138467A
S31508002140BDE8F0813846BDE8F08100BF5848000870
S3150800215070B5B84B1B78002B00F0A781012B29D14D
S31508002160FFF774FCFEF7B0F8B348FEF7F1F8B3488A
S31508002170FEF7EEF8FEF7A4F801220146B04801F092
S315080021802BFC30B1AF48FEF7E3F80120FEF7D4F890
S3150800219070BDAD48FEF7DCF8AC48FEF7D9F8AC4898
S315080021A0FEF7D6F8AB4B00221A605A600222A14B02
S315080021B01A7070BD022B40F0A880A74C04F50D726A
S315080021C04FF48071A54802F029F894F93A32002BA9
S315080021D00DDA9C48FEF7BCF80220FEF7ADF804F5C8
S315080021E00D7001F0C5FE0022924B1A7070BD0028D2
S315080021F02DD09A48002200F5C071FFF7E5FEB0F130
S31508002200FF3F0CD18F48FEF7A3F80320FEF794F89A
S315080022108B4801F0ADFE0022864B1A7070BD00286F
S3150800222015DD8C4B5B6833B98A4B8C4AD2F8802112
S315080022301A6058600BE0894AD2F8802185490968F6
S315080022408A423CBF83490A601844824B5860824BD5
S31508002250D3F83C22D3F840329A4240F02681002136
S31508002260774801F08FFE60B17648FEF771F80420D2
S31508002270FEF762F8724801F07BFE00226D4B1A7079
S3150800228070BD7148FEF764F87548FEF761F8754C3D
S31508002290704D21466868FFF7D7FD2046FEF758F8C7
S315080022A07148FEF755F82E682146300EFFF7BCFD3B
S315080022B0A11CC6F30740FFF7B7FD211DC6F307208B
S315080022C0FFF7B2FDA11DF0B2FFF7AEFD2046FEF7FF
S315080022D03FF86648FEF73CF869682868FFF7BEFBD2
S315080022E060B95848FEF734F80520FEF725F8544833
S315080022F001F03EFE00224F4B1A7070BD5248FEF7A1
S3150800230027F803224B4B1A7070BD032B40F0CD8083
S31508002310514C04F50D724FF48071504801F07EFF60
S3150800232094F93A32002B0DDA5148FEF711F80220DB
S31508002330FEF702F804F50D7001F01AFE00223D4B77
S315080023401A7070BD00285AD0444800F5807200F50E
S31508002350C071FFF739FE0646B0F1FF3F0CD145487C
S31508002360FDF7F6FF0320FDF7E7FF354801F000FE0D
S315080023700022304B1A7070BD002840DD3E48FDF73C
S31508002380E7FF384C21463046FFF75EFD2046FDF74D
S31508002390DFFF3A48FDF7DCFF304D214695F883010B
S315080023A0FFF742FDA11C95F88201FFF73DFD211DAF
S315080023B095F88101FFF738FDA11D95F88001FFF713
S315080023C033FD2046FDF7C4FF2848FDF7C1FF05F594
S315080023D080723146D5F88001FFF73CFB60B9194891
S315080023E0FDF7B6FF0620FDF7A7FF154801F0C0FD6B
S315080023F00022104B1A7070BD1348FDF7A9FF164B43
S31508002400D3F83C22D3F840329A424ED11C48FDF705
S315080024109FFFFFF72FFBA8BB0A48FDF799FF072088
S31508002420FDF78AFF064801F0A3FD0022014B1A704A
S3150800243070BD00BFB8070020744800089848000817
S31508002440F8090020C0480008C8480008D048000815
S31508002450F4480008BC070020C40700201C0C002014
S31508002460244900087807002030490008D4490008A4
S315080024704C4900087049000894490008A449000816
S31508002480BC4900080948FDF763FF0948FDF760FFE6
S31508002490084801F06DFD0848FDF75AFF0022074B72
S315080024A01A70FDF725FFFFF76DF870BDC8480008DC
S315080024B0D8490008F8090020F0490008B8070020A4
S315080024C03AB101388A1811F8013B00F8013F9142E8
S315080024D0F9D17047CA7E8B7E43EA02230278032A23
S315080024E005D1487D0A7D42EA002243EA024318469E
S315080024F0704700BF00F10B010023DA0142EA5303DB
S3150800250010F8012B134403F0FF038842F5D118464F
S31508002510704700BF10B5044601230A4600F134018E
S315080025204078FEF7F7F980BB94F8332294F83232F4
S3150800253043EA02231BB2184A934228D194F86D1035
S3150800254094F86C20130443EA016294F86A30134342
S3150800255094F86B2043EA022323F07F430F4A934201
S3150800256017D094F8890094F888301B0443EA006071
S3150800257094F88630034394F8870043EA002020F055
S315080025807F43981A18BF012010BD032010BD0220F2
S3150800259010BD002010BD00BF55AAFFFF46415400DC
S315080025A0037943B32DE9F0410446056B00F134077E
S315080025B001232A4639464078FEF7F4F9E8B900239C
S315080025C02371636A9D421BD3E26913449D421AD262
S315080025D0E678012E1AD94FF00108E3691D444346EF
S315080025E02A4639466078FEF7DDF9013E012EF4D118
S315080025F00020BDE8F081002070470120BDE8F08189
S315080026000020BDE8F0810020BDE8F0810020BDE88B
S31508002610F08100BF70B5036B8B420FD00D460446A0
S31508002620FFF7BEFF064658B901232A4604F13401CE
S315080026306078FEF76FF928B9256304E0002602E002
S31508002640012600E00126304670BD00BF90B108B5EE
S3150800265003688BB1197889B1D988828891420FD1DC
S315080026605878FEF74DF900F00100002814BF032042
S31508002670002008BD09207047092008BD092008BDAB
S31508002680092008BDF8B504682378303B092B00F209
S315080026908D8165783A2D40F08981023404600020E6
S315080026A00860002B40F05A81C94B1C68002C00F0CA
S315080026B0578115460C60237883B16078FEF720F9B8
S315080026C010F0010F0AD1002D00F04C8100F0040033
S315080026D0C0B200280CBF00200A20F8BD00202070D8
S315080026E06070FDF789FF10F0010F40F03D811DB1C4
S315080026F010F0040F40F03A8100212046FFF70AFF48
S31508002700012817D194F8F631002B00F0318194F89E
S31508002710FD2194F8FC311B0443EA026394F8FA514C
S315080027202B4394F8FB5143EA052529462046FFF733
S31508002730F1FE00E00025032800F01C81002840F087
S315080027401B8194F8402094F83F3043EA02231BB2D9
S31508002750B3F5007F40F0128194F84B0094F84A30A4
S3150800276053EA00200DD194F85B2094F85A301B04E4
S3150800277043EA026394F85800034394F8590043EA7D
S315080027800020E06194F84470E7707B1EDBB2012BF1
S3150800279000F2F68094F84130A370002B00F0F28026
S315080027A05A1E1A4240F0F08094F8466094F8452084
S315080027B042EA0626268116F00F0F40F0E78094F8C5
S315080027C0481094F8472052EA01220DD194F8571080
S315080027D094F85620120442EA016194F854200A43F8
S315080027E094F8551042EA012294F843E094F842100E
S315080027F051EA0E2100F0CC8000FB07F701EB161C0E
S31508002800BC446245C0F0C680CCEB0202B2FBF3F3CF
S31508002810002B00F0C18040F6F57E734594BF4FF05B
S31508002820010E4FF0020E4FF6F572934200F2C18088
S315080028300233A36125622944616205EB0C02E26258
S31508002840BEF1030F19D1002E40F0A88094F863104A
S3150800285094F86220120442EA016194F860200A435F
S3150800286094F8611042EA0122A2629B0003F2FF1368
S31508002870B0EB532FC0F09480BAE0002E00F092809F
S315080028803944A162BEF1020F0FBF5B0003EB43029E
S3150800289003F0010303EB5203A4E094F8332294F8FF
S315080028A0323243EA02231BB24A4A934242D194F88F
S315080028B0372094F836301B0443EA026294F8343021
S315080028C0134394F8352043EA0223434A934234D10A
S315080028D094F81B2294F81A321B0443EA026294F80D
S315080028E01832134394F8192243EA02233B4A9342C7
S315080028F026D194F8232294F822321B0443EA026272
S3150800290094F82032134394F8212243EA0223E36021
S3150800291094F81F2294F81E321B0443EA026294F8C4
S315080029201C32134394F81D2243EA022323614FF015
S31508002930030E07E04FF0030E04E04FF0030E01E02C
S315080029404FF0030E84F800E0254A138801339BB242
S315080029501380E380002020632071F8BD0B20F8BDAA
S315080029600C20F8BD0020F8BD0320F8BD0A20F8BDEC
S315080029700D20F8BD0120F8BD0D20F8BD0D20F8BDCD
S315080029800D20F8BD0D20F8BD0D20F8BD0D20F8BDB1
S315080029900D20F8BD0D20F8BD0D20F8BD0D20F8BDA1
S315080029A00D20F8BD0D20F8BD0D20F8BD00230B60E5
S315080029B07AE60233A36125622944616205EB0C02BB
S315080029C0E26240E74FF0FF3323610023E360B9E793
S315080029D0A40F002055AAFFFF52526141727241614D
S315080029E0A00F002003F2FF13B0EB532FDCD3E9E767
S315080029F04FF0FF3323610023E360637194F8652089
S31508002A0094F8643043EA02222A446261012304F1FD
S31508002A1034016078FDF77EFF00283FF43EAF4FF0A3
S31508002A20030E8FE72DE9F84301F109020369002B2C
S31508002A3067D0446994F80CC02378202B20D025460B
S31508002A4001F111064FF0E5080CF0080E5FFA8EFE4C
S31508002A5003E015F8013F202B14D0052B0AD0BEF150
S31508002A60000F08D0A3F14107FFB2192F03D820336E
S31508002A70DBB200E0434602F8013BB242E9D102E08C
S31508002A80164600E01646237A202B1ED0771C2E23E6
S31508002A903370237A202B1AD004F1080E321D0CF05D
S31508002AA0100C5FFA8CF503E01EF8013F202B10D0BE
S31508002AB035B1A3F14106F6B2192E9CBF2033DBB21D
S31508002AC007F8013BBA42EFD104E0324602E03A4643
S31508002AD000E03A46E37A0B72E67FA57F2B0443EAC9
S31508002AE00665237F2B43657F43EA05230B60657ED6
S31508002AF0237E43EA05238B80E57DA37D43EA0523F0
S31508002B00CB80002313708F6967B3CB6953B303690E
S31508002B10EBB1028C4FF6FF739A421AD0D0F81C809C
S31508002B20B8F80000B8B10D467E1E0024A1464946F5
S31508002B3001F0CEFB88B1EB69013BA3420FD9013402
S31508002B4006F8010F38F814000028F0D108E0002430
S31508002B5006E0002404E0002402E0002400E000244B
S31508002B6000233B55BDE8F88310B50446FFF718FD6A
S31508002B700346002852D12378032B47D16379002BCB
S31508002B8044D00023236304F1340104F50D700B4689
S31508002B90002203F8012B8342FBD1552384F83232F5
S31508002BA0AA2384F83332522384F8343084F8353033
S31508002BB0612384F83630412284F83720722084F85D
S31508002BC0180284F8190284F81A2284F81B32236939
S31508002BD084F81C321A1284F81D221A0C84F81E2254
S31508002BE01B0E84F81F32E36884F820321A1284F820
S31508002BF021221A0C84F822221B0E84F82332012380
S31508002C0062696078FDF7CEFE0023637100221146E3
S31508002C106078FDF71FFF031C18BF0123184610BD77
S31508002C2002398369023B99423DBF8378C06A01FB3A
S31508002C3003000020704700BF01295ED9F8B58369F3
S31508002C4099425CD20C4605460378022B28D0032B02
S31508002C5037D0012B55D101EB5107416A01EB5721BA
S31508002C60FFF7D8FC00284FD1C7F308032B4493F885
S31508002C7034600137696A01EB57212846FFF7CAFC19
S31508002C80002844D1C7F30807E81990F8340046EA43
S31508002C90002014F0010F14BF0009C0F30B00F8BDA3
S31508002CA0416A01EB1421FFF7B5FC98BB610001F4FA
S31508002CB0FF716B1893F8350093F8343043EA002017
S31508002CC0F8BD416A01EBD411FFF7A4FC28BBA100AB
S31508002CD001F4FE716A1892F8370092F836301B0430
S31508002CE043EA006392F8350043EA00200D4495F85C
S31508002CF03430184320F07040F8BD01207047012099
S31508002D00F8BD4FF0FF30F8BD4FF0FF30F8BD4FF07B
S31508002D10FF30F8BD4FF0FF30F8BD4FF0FF30F8BD7B
S31508002D2070B505460C46C1808168012938D003680C
S31508002D309A69914236D271B91A78032A01D1996AE9
S31508002D4049B90022EA601A89A2422DD99B6A03EB87
S31508002D5014132B611BE09E783601B44210D3286801
S31508002D60FFF76AFF0146B0F1FF3F1FD001281FD9C0
S31508002D702B689B6998421DD2A41BA4B2A642EED921
S31508002D80E9602868FFF74CFF00EB141028612B68F0
S31508002D90343304F00F0403EB44146C61002070BD57
S31508002DA0022070BD022070BD022070BD012070BDDA
S31508002DB0022070BD022070BD2DE9F04101297BD9A2
S31508002DC0836999427AD215460C4606460378022B41
S31508002DD03BD0032B4AD0012B66D101EB5108416A3F
S31508002DE001EB5821FFF716FC0746002861D1C8F306
S31508002DF0080314F0010F15D0334493F8342002F079
S31508002E000F0242EA051283F8342008F1010801236B
S31508002E103371716A01EB58213046FFF7FBFB002836
S31508002E2044D14DE0334483F8345008F101080123B6
S31508002E303371716A01EB58213046FFF7EBFBB8BBDB
S31508002E4043E0B04488F8342033E0416A01EB1421AA
S31508002E50FFF7E0FB074660BB610001F4FF717318DA
S31508002E6083F834502A1283F8352022E0416A01EBB0
S31508002E70D411FFF7CFFB0746D8B9A10001F4FE71BC
S31508002E80731893F837201206314402F070422A4329
S31508002E9081F83420111283F83510110C83F8361096
S31508002EA0120E83F8372004E0022702E0074600E006
S31508002EB007460123337114E0022712E0022710E0C7
S31508002EC0C8F30808C5F30712BBE7C8F3080806EBFA
S31508002ED0080393F8343023F00F03C5F303221A438B
S31508002EE0AFE73846BDE8F081F8B505460F4631B973
S31508002EF0C6686EB183699E4228BF012609E0FFF7BE
S31508002F009BFE01283BD9AB69984244D33E4600E074
S31508002F10012634460134AB699C4202D3012E30D9CE
S31508002F20022421462846FFF787FE38B1B0F1FF3F55
S31508002F3029D001282AD0B442ECD129E06FF070429A
S31508002F4021462846FFF738FF034690B937B122468F
S31508002F5039462846FFF730FF034650B9EC602B691F
S31508002F60B3F1FF3F16D0013B2B6101236B7120465D
S31508002F70F8BD012B0CBF4FF0FF300120F8BD012032
S31508002F80F8BD0020F8BD4FF0FF30F8BD0120F8BDB0
S31508002F900020F8BD2046F8BD2DE9F843C488013461
S31508002FA0A4B2002C6DD00369002B6DD00E460546E1
S31508002FB014F00F075CD101330361C16821B90368B6
S31508002FC01B89A34263D953E000688378013B13EA5F
S31508002FD014134DD1FFF730FE804601285AD9B0F1B7
S31508002FE0FF3F5AD02868836998453AD3002E57D0B0
S31508002FF0E968FFF779FF8046002854D0012855D0A4
S31508003000B0F1FF3F55D02868FFF7CAFA002853D118
S315080030102B6803F1340203F50D73002102F8011B36
S315080030209342FBD12E6841463046FFF7F9FD3063DF
S3150800303000264FF001090BE083F804902868FFF793
S31508003040AFFA013600283AD12A68136B01331363A5
S315080030502B689978F2B29142EED816461A6B961BEF
S315080030601E63C5F80C8041462868FFF7D9FD28611C
S31508003070EC802B68343303EB47136B610020BDE803
S31508003080F8830420BDE8F8830420BDE8F88304200B
S31508003090BDE8F8830220BDE8F8830120BDE8F8837F
S315080030A00420BDE8F8830720BDE8F8830220BDE8C0
S315080030B0F8830120BDE8F8830120BDE8F8830120E4
S315080030C0BDE8F8832DE9F04F85B005460021FFF7E6
S315080030D027FE002840F093804FF0FF0A5746D04657
S315080030E04FF6FF7929692868FFF794FA002840F017
S315080030F087806C692678002E00F08380E37A03F0D7
S315080031003F02E52E6CD013F0080F02D00F2A69D1C2
S3150800311001E00F2A4AD1D5F81CB0BBF1000F66D0E2
S3150800312016F0400F06D094F80DA006F0BF06EB88FF
S315080031302B8403E0B74218BF474658D1637B0193F7
S31508003140534551D1237823F04003013B03EB430257
S3150800315003EB82030293344F07F10D0A012017F897
S31508003160012BA3185978A35C43EA012380B11846BA
S3150800317001F0D0F80390029BFE2B4DD85A1C029200
S315080031803BF8130001F0C6F8039B834244D101E0E3
S315080031904B4541D15745E2D1237813F0400F36D03D
S315080031A0A8B3029B3BF813308BB335E027B920460A
S315080031B0FFF7A0F9824526D0A5F82090AB69DA7A00
S315080031C012F0010F12D104F10B0001E0A0421CD04D
S315080031D014F8011B13F8012B9142F7D0474606E075
S315080031E0474604E0474602E0474600E047460021D6
S315080031F02846FFF7D1FE00283FF474AF10E00FE031
S315080032000EE004200CE000200AE0002008E0013E61
S31508003210F7B2DDF804A0EAE7DDF804A04746E6E7DA
S3150800322005B0BDE8F08F00BFB04A00082DE9F04FA1
S3150800323083B005468B460B782F2B01D05C2B01D12A
S315080032400BF1010B0023AB609BF800301F2B09D84C
S3150800325000212846FFF764FD034600226A6157E10C
S315080032609B46FFE7D8465B4613F8010B2F28F7D095
S315080032705C2808BF9B46F5D0EE6980B21F2840F24D
S315080032801E812F2800F021815C2800F02181B71EBD
S315080032900124A1460AE02F2800F01C815C2800F0D2
S315080032A01981B3F5807F00F029811C46494601F053
S315080032B00FF80146002800F021817F2809D8222826
S315080032C000F0E280944A12F8013F13B19842FAD10D
S315080032D0DAE027F8021F631C1BF8010F1F28DAD84B
S315080032E0EFE0002C00F0D08006EB440232F8023DF5
S315080032F0202B01D02E2B02D1013CF7D1C4E0002CA3
S3150800330000F0FC806000002326F81430AB6903F156
S315080033100B01202203F8012B9942FBD1B11E002391
S3150800332000E0013331F8022F202AFAD02E2AF8D0ED
S31508003330002B00F0D38047F00307CFE0013C06D10D
S315080033404FF0080A4FF00009CDF8049004E032F86F
S31508003350021D2E29F2D1F3E703F1010836F813000E
S3150800336000285ED0202803D02E2805D1A04503D0FA
S3150800337047F003074346EFE7D14502D2A04519D1E6
S31508003380BEE0BAF10B0F06D147F00307AB691A780E
S31508003390E52A56D14AE0A04502D047F0030740D8AF
S315080033A0019B9B00DBB2019323464FF00B0A4FF0BB
S315080033B00809D1E77F2840F29880002100F088FFAD
S315080033C00346002800F0A180544A134413F8801CD1
S315080033D088B247F0020748B12B2907D0504A12F89D
S315080033E0013F002B00F083808B42F8D147F003079A
S315080033F05F200FE0019B43F0020301930AE0A0F16E
S3150800340061039BB2192B05D8019B43F00103019375
S31508003410203880B2AB6903F80900434609F101096F
S315080034209AE7AB691A78E52A04D101E04FF00B0A4E
S3150800343005221A70BAF1080F03D1019B9B00DBB273
S315080034400193019A02F00C030C2B03D002F003023D
S31508003450032A01D147F0020717F0020F0AD1019A91
S3150800346002F00302012A08BF47F01007042B08BF21
S3150800347047F00807AB69DF722846FFF723FEAB69FA
S31508003480DA7A034660B101E0062341E004283FD119
S3150800349002F00402D2B2002A14BF0346052337E01D
S315080034A012F0040F34D16969CB7A13F0100F04D0E7
S315080034B02868FFF70FF8A860D4E6052328E000245B
S315080034C0012308EB030B04270BE70024012301E083
S315080034D00024012308EB030B002702E7811E72185C
S315080034E0715A2E293FF42CAF28E7014674E7A0F15C
S315080034F041039BB2192B7FF67DAF80E7062307E0D1
S31508003500BAF10B0F7FF44CAF3EE747F002076DE7C1
S31508003510184603B0BDE8F08F1C4A0008304A000878
S31508003520284A00082DE9F84F044688464FF0FF0A56
S315080035305646042557464FF6FF796DE02068FFF793
S3150800354069F8054600286BD160690378002B71D0AD
S31508003550E52B54D02E2B54D0C27A02F03F02082A0B
S3150800356014BF0021012141454DD10F2A3ED113F048
S31508003570400F06D090F80DA003F0BF03E28822841E
S3150800358003E09E4218BF3E4640D190F80DE0D6456E
S315080035903BD1D4F81CA0027802F03F02013A02EBB4
S315080035A0420502EB8505264901F10D0C012611F8A5
S315080035B0012B00EB020B9BF801B0825C42EA0B225E
S315080035C036B1FE2D33D82AF815201646013501E006
S315080035D04A452CD18C45EAD1027812F0400F22D008
S315080035E0FE2D24D800222AF815201CE01EB9FEF765
S315080035F081FF824520D04FF6FF7323841CE03E46A8
S3150800360004E03E4602E03E4600E03E4600212046F3
S31508003610FFF7C2FC054618B9216900298ED15DB1AC
S315080036200023236108E0013BDEB2F246EEE7F246EC
S315080036303E46EBE70425F3E72846BDE8F88F00BFCA
S31508003640B04A00082DE9F0410446C588018C4FF6BA
S31508003650FF73994208BF2946FFF762FB0346D0B9B4
S31508003660E52701264FF0000821692068FEF7D2FFFA
S31508003670034668B96269177022681671E288AA4219
S3150800368009D241462046FFF787FC03460028EBD0BF
S31508003690042B08BF02231846BDE8F081012928D962
S315080036A02DE9F04104460E468369994224D2002743
S315080036B04FF0010831462046FFF7BEFA0546E8B145
S315080036C001281DD0B0F1FF3F1CD03A4631462046AE
S315080036D0FFF772FB0246B0B92369B3F1FF3F03D087
S315080036E00133236184F805802E46A369AB42E1D8ED
S315080036F009E0022210467047022204E0002202E096
S31508003700022200E001221046BDE8F08170B582B0C1
S31508003710054616461C460B22FEF7D2FE052C09D98D
S31508003720E30343EA540436F8023B1C44A4B2338844
S31508003730002BF5D102A8072204F00F0101F130038E
S31508003740392B88BF01F13703013A00F8013D2409F6
S31508003750F2D17E2102AB134403F8081C62B12B7820
S31508003760202B0BD02946002301339A4207D011F8A3
S31508003770010F2028F8D102E0002300E00023E81812
S3150800378020240133072A05D802A9114411F8081C78
S31508003790013200E0214600F8011B072BF1D902B0DF
S315080037A070BD00BF2DE9F04F87B004468769C6692A
S315080037B00C2239460DEB0200FEF782FE9DF8173003
S315080037C013F0010F1DD00023FB72E36101252B4680
S315080037D0324603A93846FFF799FF2046FFF772FCE1
S315080037E028B90135ADB2642DF1D10720DAE0642D90
S315080037F000F0BF80042840F0BE809DF81730FB72A9
S31508003800E6619DF8173013F0020F13D033883BB1E9
S31508003810002301339BB236F81320002AF9D100E0C1
S3150800382000231933614D85FB0325DB17C3EBA5057B
S31508003830ADB200E0012500212046FFF771FA0346E4
S31508003840002840F0AE800026012721692068FEF78F
S31508003850E1FE0346002840F0A48063691B78E52B47
S3150800386000D01BB90136B54201D185E0002639469C
S315080038702046FFF791FB03460028E6D091E0E18851
S31508003880491B89B22046FFF74BFA0346002840F049
S315080038908680A069FEF72EFE009000270197216911
S315080038A02068FEF7B7FE0346002878D1D4F81C90A6
S315080038B060695FFA85FB9DF8003043734FF00F038C
S315080038C0C37207738776C7760BF1FF3303EB4301A1
S315080038D003EB8101364A02F10D08019B4FF6FF768C
S315080038E04FF0FF0AB3424BD001F1010E39F81130FF
S315080038F01178435401444FEA132C81F801C013B9D7
S315080039007146334600E0714601329045EAD14FF6DA
S31508003910FF72934202D039F811300BB94BF0400BC5
S3150800392080F800B0236801221A7139462046FFF74D
S3150800393033FB0346002832D1013DADB2002DAED18E
S3150800394026E0636903F12001002203F8012B99425E
S31508003950FBD10B22A1696069FEF7B2FD6269A36912
S31508003960DB7A03F018031373236801221A71002007
S3150800397018E0072016E015E0013DADB245B17EE737
S3150800398092F800E000F80EA086448EF801A0BBE786
S3150800399021692068FEF73EFE0028D2D002E01846CC
S315080039A000E0184607B0BDE8F08F00BF4FECC44EE4
S315080039B0B04A000858B9074B1B680BB100221A70A9
S315080039C009B100230B70034B1960002070470B20C8
S315080039D0704700BFA40F00202DE9F0438FB0019176
S315080039E0002800F08980044615460023036002F08B
S315080039F01E0205A901A8FEF745FE00287ED105F09E
S31508003A001F0702AB0B93514B0C93019905A8FFF7BF
S31508003A100DFC0A9E0346002871D1002E7AD172E069
S31508003A20042B7FD105A8FFF7BDFE47F008070A9EBD
S31508003A30034638B186E0F37A13F0110F7BD115F0FF
S31508003A40040F7AD117F0080F39D0FDF737F9B0739C
S31508003A500312F373030C3374000E70740025F572A9
S31508003A6035777577B577F577DDF8148031464046B2
S31508003A70FEF730FDB576F57635757575012388F848
S31508003A8004300546C8B1D8F8309001464046FFF7DD
S31508003A9005FE0346002855D10598013DC5604946EF
S31508003AA0FEF7B8FD48B14EE015F0020F02D013F04C
S31508003AB0010F44D115F0080F01D047F02007059BE8
S31508003AC01B6BE3612662A771059D31462846FEF702
S31508003AD001FD2061F17FB27F130443EA0162337F5F
S31508003AE01343727F43EA0223E3600020A060A061CB
S31508003AF02560EB88A38026E0092024E023E015F062
S31508003B001C0F0BD08CE715F01C0F18BF062309D124
S31508003B10062303E015F01C0F8DD107E0002BD2D049
S31508003B20184610E047F008070A9EF7E7F37A13F0FD
S31508003B30100F06D1B8E7072005E0082003E00723A1
S31508003B4000E0042318460FB0BDE8F083A00D00205E
S31508003B502DE9F04F83B0044689461546984600235A
S31508003B60C8F80030FEF772FD002840F0B980A37946
S31508003B7013F0800F40F0B58013F0010F00F0B3800A
S31508003B80E368A6689E1BAE4228BF2E46002E00F0AC
S31508003B90AC8004F124030193A268C2F30803002B46
S31508003BA040F0828020688378013B03EA522313F0B1
S31508003BB0FF0717D10AB9206902E06169FFF73CF8E7
S31508003BC0012805D8A37963F07F03A37102208DE04D
S31508003BD0B0F1FF3F05D1A37963F07F03A3710120FC
S31508003BE084E06061D4F800A061695046FFF718F8D0
S31508003BF0054628B9A37963F07F03A371022075E00F
S31508003C003D445FEA562B28D09AF8023007EB0B02A0
S31508003C109A4288BFC7EB030B5FFA8BF32A464946DD
S31508003C209AF80100FCF776FE28B1A37963F07F03C2
S31508003C30A37101205AE0A37913F0400F0AD0A069B6
S31508003C40401B834506D94FF40072019909EB4020C1
S31508003C50FEF736FC4FEA4B2534E0A269954222D09E
S31508003C60A37913F0400F10D0012301999AF80100A7
S31508003C70FCF798FE28B1A37963F07F03A3710120AE
S31508003C8034E0A37923F04003A371206801232A4670
S31508003C9001994078FCF73EFE28B1A37963F07F03CB
S31508003CA0A371012022E0A561A168C1F30801C1F54D
S31508003CB00075B54228BF354621442A462431484670
S31508003CC0FEF7FEFBA944A3682B44A360D8F800308E
S31508003CD02B44C8F80030761B7FF45EAF002005E061
S31508003CE004E0022002E0072000E0002003B0BDE85F
S31508003CF0F08F00BF2DE9F04F83B00446894616467B
S31508003D0098460023C8F80030FEF7A0FC002840F0CB
S31508003D10D380A37913F0800F40F0CF8013F0020F01
S31508003D2000F0CD80E368F34280F0BB80002E00F0FF
S31508003D30B88004F124030193A268C2F30803002B98
S31508003D4040F0918020688378013B03EA522313F000
S31508003D50FF0721D13AB9236963B90021FFF7C4F8EF
S31508003D600346206103E06169FFF7BEF80346002BAE
S31508003D7000F09780012B05D1A37963F07F03A37127
S31508003D8002209DE0B3F1FF3F05D1A37963F07F03DD
S31508003D90A371012094E06361A37913F0400F11D059
S31508003DA020680123A26901994078FCF7FBFD28B138
S31508003DB0A37963F07F03A371012081E0A37923F03F
S31508003DC04003A371D4F800A061695046FEF728FFA6
S31508003DD0054628B9A37963F07F03A37102206FE033
S31508003DE03D445FEA562B28D09AF8023007EB0B02BF
S31508003DF09A4288BFC7EB030B5FFA8BF32A464946FC
S31508003E009AF80100FCF7CEFD28B1A37963F07F0389
S31508003E10A371012054E0A169491B8B450AD94FF4C7
S31508003E20007209EB41210198FEF74AFBA37923F0BA
S31508003E304003A3714FEA4B2527E0A3699D4211D0A1
S31508003E40A268E3689A420DD201232A4601999AF894
S31508003E500100FCF75FFD28B1A37963F07F03A37126
S31508003E6001202DE0A561A068C0F30800C0F5007523
S31508003E70B54228BF354620442A4649462430FEF72F
S31508003E801FFBA37943F04003A371A944A3682B44FD
S31508003E90A360D8F800302B44C8F80030761B7FF4AE
S31508003EA04BAFA368E268934288BFE360A37943F007
S31508003EB02003A371002003E002E0022000E00720AF
S31508003EC003B0BDE8F08F00BF38B50446FEF7BEFB69
S31508003ED0002846D1A37913F0200F43D013F0400FE2
S31508003EE00DD020680123A26904F124014078FCF76B
S31508003EF059FD002838D1A37923F04003A371E1695D
S31508003F002068FEF787FB88BB256AEB7A43F0200317
S31508003F10EB72E3682B77E3681B126B77E389AB7761
S31508003F20E37BEB772369AB761A12EA761B0C2B75C3
S31508003F301B126B75FCF7C2FEA8750312EB75030C12
S31508003F402B76000E68760023AB74EB74A37923F006
S31508003F502003A371236801221A712068FEF704FE64
S31508003F6038BD38BD002038BD012038BD38BD00BF7A
S31508003F7010B50446FFF7A8FF034608B900222260D9
S31508003F80184610BD70B504460D46FEF75FFB0028BF
S31508003F9040F0BC80A37913F0800F40F0B880E26847
S31508003FA0AA4205D203F00203DBB2002B08BF15466E
S31508003FB0A3680022A260002D00F0AB8020688678F6
S31508003FC076026BB1013B6A1EB2FBF6F2B3FBF6F161
S31508003FD08A4205D372421340A360ED1A616917E05D
S31508003FE02169A1B9FEF780FF0146012805D1A37909
S31508003FF063F07F03A371022070BDB0F1FF3F05D1C6
S31508004000A37963F07F03A371012070BD206161610C
S31508004010002940D0B5422BD9A37913F0020F05D059
S315080040202068FEF761FF014620B920E02068FEF708
S3150800403003FE0146B1F1FF3F05D1A37963F07F0383
S31508004040A371012070BD012903D923689B69994290
S3150800405005D3A37963F07F03A371022070BD616164
S31508004060A3683344A360AD1BAE42D5D300E0354602
S31508004070A3682B44A360C5F3080373B12068FEF751
S31508004080CFFD28B9A37963F07F03A371022070BD21
S3150800409000EB552502E0002500E00025A368C3F3E0
S315080040A0080343B3A269954225D0A37913F0400FBC
S315080040B011D02068012304F124014078FCF772FC32
S315080040C028B1A37963F07F03A371012070BDA3799A
S315080040D023F04003A371206801232A4604F1240132
S315080040E04078FCF717FC28B1A37963F07F03A37126
S315080040F0012070BDA561A368E26893420BD9E3600D
S31508004100A37943F02003A371002070BD70BD02207F
S3150800411070BD002070BD002070BD00BF30B58FB0E7
S3150800412001900D46002205A901A8FEF7ABFA044640
S3150800413088B902AB0B93094B0C93019905A8FFF7B5
S3150800414075F8044638B90A9B23B1294605A8FEF72F
S3150800415069FC00E0062420460FB030BDA00D002003
S3150800416030B599B0019001220FA901A8FEF78AFA85
S31508004170044600284CD103AB1593274B1693019997
S315080041800FA8FFF753F80446002841D1149959B3EC
S31508004190CC7A14F0010F29D12FE0012D35D924222C
S315080041A00FA906A8FEF78CF90895022106A8FEF7BE
S315080041B0B7FD044660BB002106A8FFF7B3F904461D
S315080041C028B3042824D10FA8FFF73CFA0446F8B907
S315080041D02DB129460F98FFF761FA0446C0B90F9822
S315080041E0FEF7C2FC044613E0062400E007240F98F5
S315080041F0FEF770F905465CB9E5E70F98FEF76AF928
S31508004200054614F0100FC8D1DDE7022400E00724A4
S31508004210204619B030BD00BFA00D00202DE9F041A1
S3150800422082B080461746054600244E1E12E06B46AD
S31508004230012201A93846FFF78BFC009B012B0DD103
S315080042409DF804300D2B05D06A1C2B7001340A2BFF
S3150800425003D01546B442EADB00E0154600232B706E
S315080042609C4214BF4046184602B0BDE8F08100BF24
S3150800427030B583B004460D460A2802D10D20FFF753
S31508004280F7FF8DF8004001AB012269462846FFF783
S3150800429031FD019B012B0CBF01204FF0FF3003B00D
S315080042A030BD00BF037883B170B50E460546441C81
S315080042B031461846FFF7DCFFB0F1FF3F07D0601B19
S315080042C014F8013B002BF3D170BD0020704770BD78
S315080042D07F281BD911B9C72808D112E0FF2814D89E
S315080042E0A0F180030A4A32F813007047084A0123EE
S315080042F032F8021F814205D001339BB2802BF7D1D9
S3150800430000E000238033D8B270470020704700BF12
S31508004310A04C0008612809D008490022013231F86A
S31508004320023F4BB18342F9D108B904E00022044B9D
S3150800433033F8120070470020704700BFC04A0008D3
S31508004340A04D0008034BFE22DA7018710222A3F86A
S3150800435044207047A80F0020054B00221A709A6463
S3150800436083F84320A3F844209A705A70704700BF18
S31508004370A80F0020024B1878003018BF012070479C
S31508004380A80F00200022024B83F84320704700BF85
S31508004390A80F002038B50378FF2B22D1FDF7B2FD10
S315080043A018B91020FFF7CEFF61E1AD4C002363700A
S315080043B001252570FF22E270102222716371FDF734
S315080043C0EDFCA071FDF7FCFCE071FDF7F9FC000AB5
S315080043D020726572A5720823A4F84430FDF736FBEF
S315080043E045E104469E4A1278012A40F06081C93B9D
S315080043F0352B00F23981DFE813F0C00037013701A9
S315080044002F01370137012601DB00150105013701A8
S3150800441037013701370137013701370137013701CE
S3150800442037013701370137013701370137013701BE
S3150800443037013701370137013701370137013701AE
S315080044403701370137013701370137013701760060
S31508004450510036006D0037013701370192003701E8
S31508004460A400A800B6004578FDF798FC01388542F7
S3150800447003DD2220FFF766FFF9E0794D6278A96C23
S31508004480281DFDF79BF8FF23EB706378AA6C13448D
S31508004490AB6463780133A5F84430E8E04578FDF766
S315080044A07DFC0138854203DD2220FFF74BFFDEE065
S315080044B061686B4DA9646278281DFDF77FF8FF23B4
S315080044C0EB706378AA6C1344AB6463780133A5F880
S315080044D04430CCE0624BFF22DA7042689A640122CB
S315080044E0A3F84420DDE05E4BFF22DA709A6C406840
S315080044F040B11044002312F8011B0B44DBB2904272
S31508004500F9D100E00023564AC2F807300123137197
S315080045100023537193710823A2F84430C1E0504B2D
S31508004520FF22DA704F4A9A6400221A715A719A71F8
S315080045300721D9711A725A729A720822A3F844206E
S31508004540AFE00020FFF7FEFE91E0454BFF22DA7050
S3150800455000221A71597859719A71DA711A720622FB
S31508004560A3F844209DE03E4B00221A705A70FF22A1
S31508004570DA700122A3F8442093E0394B9D6CFDF7CD
S315080045800DFC621C411E2846FDF764FA18B9312055
S31508004590FFF7D8FE6BE0324CFF23E370FDF7FEFB16
S315080045A00138A36C0344A3640123A4F8443078E0DB
S315080045B04578FDF7F3FB0238854203DD2220FFF735
S315080045C0C1FE54E0264BFF22DA700122A3F84420EC
S315080045D0617839B9FDF74EFA002848D13120FFF73E
S315080045E0B1FE44E0A21C1E4B986CFDF733FA18B9CD
S315080045F03120FFF7A7FE3AE0194A6378916C0B441D
S31508004600936434E0164CFF23E37000252571657129
S31508004610FDF7C4FBA071E571257265720723A4F83E
S3150800462044303EE041680E4B986CFDF717FA18B90E
S315080046303120FFF787FE1AE0094BFF22DA700122C4
S31508004640A3F844202DE0FCF79DFF054BFF22DA7006
S315080046500122A3F8442024E03120FFF773FE06E088
S31508004660A80F0020804F00082020FFF76BFE104B94
S3150800467093F84330012B02D11020FFF763FE0C4B51
S31508004680B3F94410002912DD0948012380F84330A4
S3150800469089B20330FDF76CFB38BD054BB3F94410FE
S315080046A0F2E7034B93F84330012BF6D1E4E738BD24
S315080046B0A80F002008B5074B044613B10021AFF335
S315080046C00080054B1868836A03B19847204600F0B6
S315080046D033F800BF000000008C5000080E4B70B580
S315080046E01E460E4C0025E41AA410A54204D056F81E
S315080046F0253098470135F8E700F020F8084B094CB3
S315080047001E46E41AA4100025A54204D056F8253002
S3150800471098470135F8E770BD7C0000207C00002032
S315080047207C0000208000002003460244934202D009
S3150800473003F8011BFAE77047FEE70000F8B500BF6B
S31508004740F8BC08BC9E467047F8B500BFF8BC08BC64
S315080047509E4670472F64656D6F70726F675F7374DE
S315080047606D3332663230372E73726563000000008F
S315080047702F626F6F746C6F672E7478740000000078
S315080047802E2E5C2E2E5C2E2E5C2E2E5C536F757292
S3150800479063655C41524D434D335F53544D33324646
S315080047A0325C63616E2E6300050206020603070388
S315080047B00803090309040A040B040C040C050D0577
S315080047C00E050F050F061006100710080000080052
S315080047D0100018002000280030003800400048006B
S315080047E05000580000800008004000000200000049
S315080047F000C0000800400000030000000000010897
S315080048000000010004000000000002080000020089
S315080048100500000000000408000002000600000071
S315080048200000060800000200070000002E2E5C2E7D
S315080048302E5C2E2E5C2E2E5C536F757263655C4162
S31508004840524D434D335F53544D333246325C756196
S3150800485072742E63000000002E2E5C2E2E5C2E2E07
S315080048605C2E2E5C536F757263655C66696C652E8B
S31508004870630000004669726D776172652075706421
S3150800488061746520726571756573742064657465F5
S31508004890637465640A0D00004F70656E696E672063
S315080048A06669726D776172652066696C6520666FE8
S315080048B0722072656164696E672E2E2E00000000F4
S315080048C04552524F520A0D004F4B0A0D0000000088
S315080048D05374617274696E67207468652070726FAC
S315080048E06772616D6D696E672073657175656E6354
S315080048F0650A0D0050617273696E67206669726D8C
S31508004900776172652066696C6520746F206F6274C2
S3150800491061696E2065726173652073697A652E2EEA
S315080049202E00000045726173696E67200000000062
S315080049302062797465732066726F6D206D656D6F80
S315080049407279206174203078000000005265616435
S31508004950696E67206C696E652066726F6D20666980
S315080049606C652E2E2E4552524F520A0D000000003D
S31508004970496E76616C696420636865636B73756DEF
S3150800498020666F756E642E2E2E4552524F520A0DB2
S315080049900000000050726F6772616D6D696E672066
S315080049A00000000020627974657320746F206D65BD
S315080049B06D6F7279206174203078000057726974BF
S315080049C0696E672070726F6772616D2063686563D0
S315080049D06B73756D2E2E2E00436C6F73696E672090
S315080049E06669726D776172652066696C650A0D0085
S315080049F04669726D776172652075706461746520A9
S31508004A007375636365737366756C6C7920636F6D14
S31508004A10706C657465640A0D00000000222A3A3C31
S31508004A203E3F7C7F000000002B2C3B3D5B5D000079
S31508004A30809A90418E418F804545454949498E8FD8
S31508004A409092924F994F555559999A9B9C9D9E9F26
S31508004A5041494F55A5A5A6A7A8A9AAABAC21AEAFB3
S31508004A60B0B1B2B3B4B5B6B7B8B9BABBBCBDBEBFC0
S31508004A70C0C1C2C3C4C5C6C7C8C9CACBCCCDCECFB0
S31508004A80D0D1D2D3D4D5D6D7D8D9DADBDCDDDEDFA0
S31508004A90E0E1E2E3E4E5E6E7E8E9EAEBECEDEEEF90
S31508004AA0F0F1F2F3F4F5F6F7F8F9FAFBFCFDFEFF80
S31508004AB001030507090E10121416181C1E00000023
S31508004AC061006200630064006500660067006800B4
S31508004AD069006A006B006C006D006E006F00700064
S31508004AE07100720073007400750076007700780014
S31508004AF079007A00A100A200A300A500AC00AF00CF
S31508004B00E000E100E200E300E400E500E600E7007B
S31508004B10E800E900EA00EB00EC00ED00EE00EF002B
S31508004B20F000F100F200F300F400F500F600F800DA
S31508004B30F900FA00FB00FC00FD00FE00FF00010181
S31508004B4003010501070109010B010D010F011101FF
S31508004B5013011501170119011B011D011F0121016F
S31508004B6023012501270129012B012D012F013101DF
S31508004B703301350137013A013C013E01400142014A
S31508004B804401460148014B014D014F0151015301B2
S31508004B905501570159015B015D015F01610163011F
S31508004BA06501670169016B016D016F01710173018F
S31508004BB0750177017A017C017E019201B103B20386
S31508004BC0B303B403B503B603B703B803B903BA030B
S31508004BD0BB03BC03BD03BE03BF03C003C103C303BA
S31508004BE0C403C503C603C703C803C903CA033004FD
S31508004BF031043204330434043504360437043804E3
S31508004C0039043A043B043C043D043E043F04400492
S31508004C104104420443044404450446044704480442
S31508004C2049044A044B044C044D044E044F045104F1
S31508004C30520453045404550456045704580459049A
S31508004C405A045B045C045E045F04702171217221BE
S31508004C5073217421752176217721782179217A218A
S31508004C607B217C217D217E217F2141FF42FF43FF5D
S31508004C7044FF45FF46FF47FF48FF49FF4AFF4BFFF2
S31508004C804CFF4DFF4EFF4FFF50FF51FF52FF53FFA2
S31508004C9054FF55FF56FF57FF58FF59FF5AFF0000AC
S31508004CA0C700FC00E900E200E400E000E500E700D8
S31508004CB0EA00EB00E800EF00EE00EC00C400C500D7
S31508004CC0C900E600C600F400F600F200FB00F90091
S31508004CD0FF00D600DC00A200A300A500A7209201D1
S31508004CE0E100ED00F300FA00F100D100AA00BA00D5
S31508004CF0BF001023AC00BD00BC00A100AB00BB0088
S31508004D009125922593250225242561256225562578
S31508004D1055256325512557255D255C255B251025D9
S31508004D20142534252C251C2500253C255E255F25C4
S31508004D305A25542569256625602550256C2567253D
S31508004D4068256425652559255825522553256B253B
S31508004D506A2518250C25882584258C2590258025E7
S31508004D60B103DF009303C003A303C303B500C40361
S31508004D70A6039803A903B4031E22C603B503292272
S31508004D806122B1006522642220232123F7004822EC
S31508004D90B0001922B7001A227F20B200A025A00071
S31508004DA041004200430044004500460047004800D1
S31508004DB049004A004B004C004D004E004F00500081
S31508004DC05100520053005400550056005700580031
S31508004DD059005A002100E0FFE1FFE5FFE2FFE3FF8B
S31508004DE0C000C100C200C300C400C500C600C70099
S31508004DF0C800C900CA00CB00CC00CD00CE00CF0049
S31508004E00D000D100D200D300D400D500D600D800F7
S31508004E10D900DA00DB00DC00DD00DE0078010001E5
S31508004E2002010401060108010A010C010E01100124
S31508004E3012011401160118011A011C011E01200194
S31508004E4022012401260128012A012C012E01300104
S31508004E5032013401360139013B013D013F0141016F
S31508004E604301450147014A014C014E0150015201D7
S31508004E705401560158015A015C015E016001620144
S31508004E806401660168016A016C016E0170017201B4
S31508004E907401760179017B017D01910191039203E9
S31508004EA093039403950396039703980399039A0328
S31508004EB09B039C039D039E039F03A003A103A303D7
S31508004EC0A403A503A603A703A803A903AA0310041A
S31508004ED01104120413041404150416041704180400
S31508004EE019041A041B041C041D041E041F042004B0
S31508004EF02104220423042404250426042704280460
S31508004F0029042A042B042C042D042E042F0401043E
S31508004F100204030404040504060407040804090437
S31508004F200A040B040C040E040F046021612162219B
S31508004F3063216421652166216721682169216A2127
S31508004F406B216C216D216E216F2121FF22FF23FF2A
S31508004F5024FF25FF26FF27FF28FF29FF2AFF2BFF0F
S31508004F602CFF2DFF2EFF2FFF30FF31FF32FF33FFBF
S31508004F7034FF35FF36FF37FF38FF39FF3AFF0000A9
S31508004F804F70656E424C54000020202020202020BF
S31508004F9020202828282828202020202020202020DB
S31508004FA020202020202020202088101010101010EB
S31508004FB01010101010101010100404040404040437
S31508004FC004040410101010101010414141414141D1
S31508004FD001010101010101010101010101010101B3
S31508004FE001010101101010101010424242424242C3
S31508004FF00202020202020202020202020202020283
S31508005000020202021010101020000000000000002A
S315080050100000000000000000000000000000000082
S315080050200000000000000000000000000000000072
S315080050300000000000000000000000000000000062
S315080050400000000000000000000000000000000052
S315080050500000000000000000000000000000000042
S315080050600000000000000000000000000000000032
S315080050700000000000000000000000000000000022
S315080050800000000000000000004300001C00002093
S30908005090000000000E
S30D080050944CB1FF7F010000008A
S3150800509C01000000000000000102030401020304E1
S315080050AC0607080904000000884F000800000000E5
S315080050BC00000000000000000000000000000000D6
S315080050CC00000000000000000000000089500008E5
S315080050DC00000000000000000000000000000000B6
S315080050EC00000000000000000000000000000000A6
S315080050FC0000000000000000000000000000000096
S3150800510C000000000000000000000000A9010008D3
S3090800511C85010008F3
S70508000000F2
